:020000020000FC
:100000009FC947C20000000025C000004DC100008C
:10001000000050C1000000000000000002030406C0
:10002000080C101820304060800002030406080C01
:10003000101820304080FF000406080C10182030F3
:10004000406080A0C0000D0D0405060D050D0602E0
:10005000030302004FB662FD1EC070FF18C165FDAC
:10006000F8C00994C0919700C395C0939700C5E06C
:10007000C519B8F3D0919700CD1B98F3C8E7089441
:1000800083FDC795C4BDC52DCC2321F4C0E083FDFD
:10009000C0E8C4BD07C171FF03C09598AC98C09873
:1000A000C52D089483FDC795C4BDC09399006B7F8F
:1000B000C52DCF3F09F441C0C0919800C395C093AE
:1000C000980070FF35C09598AC98C0984FBE1895B1
:1000D0007860C091A000CC2391F0C0919800CA959F
:1000E000D091A000CD1B58F0777FC0919800D0919F
:1000F0009F00CD1B08F41CC02092980019C0959851
:10010000AC98C098C5E0CA95F1F7C0917500CA9542
:10011000C2FD09C0C1FD05C095FF949A95FDAB9A3B
:100120000EC0AD9A0CC095FFAB9A95FD949A07C08E
:100130009598AC98C0984FBE1895209299004FBEE4
:100140001895A5C0552021F095FF959A95FDC09A68
:10015000AC989DC0552009F0AC9A95FFC09895FDCC
:10016000959895C0552021F095FFC09A95FD959AD8
:1001700095FF959895FDC0988AC095FFAB9895FD21
:10018000949895FF949895FDAB98C5E0CA95F1F7C2
:10019000552021F095FF959A95FDC09AAC9877C0AF
:1001A00095FFAB9895FD9498AD98C5E0CA95F1F789
:1001B000552021F095FF959A95FDC09AAC9867C09F
:1001C000AD9895FFAB9895FD9498C5E0CA95F1F769
:1001D000552009F0AC9A95FFC09895FD959857C0A9
:1001E000AD9895FF949895FDAB98C5E0CA95F1F749
:1001F000552009F0AC9A95FFC09895FD959847C099
:1002000095FF949895FDAB98AD98C5E0CA95F1F728
:10021000552021F095FFC09A95FD959A95FF9598E8
:1002200095FDC09834C095FF949895FDAB9895FFC7
:10023000AB9895FD9498C5E0CA95F1F7552021F04B
:1002400095FFC09A95FD959A95FF959895FDC09854
:100250001EC082FF1CC0C0917500C2FD0BC0C1FD55
:1002600011C095FFAB9895FD949895FF949895FDD6
:10027000AB980DC0C1FDF5CF95FFAB9895FD949857
:10028000AD9805C0AD9895FF949895FDAB98C52D98
:10029000C095089483FDC795C4BDC0939900209272
:1002A000970064604FBE18954FB6C0E1C8BF6E7F1F
:1002B0004FBE18953FB68F7EABB7A074A211806178
:1002C000A0E0ABBFA9B7AE7FA9BF7894A0916600AC
:1002D000AA2349F0A92FAF7151F1A0916600AA9508
:1002E000A093660024C040E050E0A0B396FDA09526
:1002F000A2FD4FEF96FFA3E096FDA2E0A5BFAA27BF
:10030000A064AABF8D7FA0B396FDA095A2FD5FEF6C
:10031000451749F7A8E161FDA0936600A92FAF71C9
:1003200019F0A8E1A093660040938D008160A09130
:100330006700AA2331F0A0916700AA95A0936700F7
:1003400007C0A92FAF7121F08061AA27A064AABFBE
:1003500080FF4BC0A0918D004A2F8E7FA92FAF71D7
:10036000E1F0A091AE00A430C1F4403F08F040EFAE
:10037000A42FA295AF704A0F5091B000533069F08E
:10038000A695A69550FD01C0A69552FD03C0A41BDD
:100390004A2F03C04A0F08F44FEF4093610071FFEA
:1003A00008C0A091610050919200A51710F05093E1
:1003B00061004091AE00443029F5A0916100409168
:1003C0006300A41B70F04091CF00A40B50F0A091EB
:1003D0006300A40FA093630040F4AFEFA093630009
:1003E00004C0A0916100A093630040916300A091BC
:1003F00092004A1708F04A2FA09194004A1708F07B
:100400004A2F542EA52DA03408F06860A0916000FA
:10041000A395A093600051F0F894A9B7A160A9BF7B
:1004200084FF02C0A0E4ABBF3FBE189541E05091ED
:100430006600552331F0A92FAF7119F45A955093E6
:100440006600A0918D00A13018F0209290000DC0A0
:100450002092910020929A00A0919000AF5FA0930B
:10046000900018F0AFEFA0939000A0919300A65FCA
:1004700020F05FEF5093930002C0A0939300F89494
:10048000A9B7A160A9BF84FF02C0A0E4ABBF3FBE73
:1004900018953FB64CB55DB58F7EABB7A074A21171
:1004A0008061A0E0ABBFA9B7AE7FA9BF789481FD02
:1004B00026C096FFA2E096FDA3E0A5BF8260A0B390
:1004C00096FDA095A2FF05C040936400509365007F
:1004D00033C196FFA3E096FDA2E0A5BFAA27A064C2
:1004E000AABF8D7FA92FAF7109F417C140E0A0B357
:1004F00096FDA095A2FD11C140938D0004C196FF09
:10050000A3E096FDA2E0A5BF8D7F61FF6BC096FFC3
:10051000A2E096FDA3E0A5BFAA27A064AABF8260BF
:100520004093880050938900A09086004A19B090AB
:1005300087005B09BB24A2E0EA2EA22C483CA0E085
:100540005A0730F4A0E1BA2EE22CAAE0AA2E27C066
:100550004836A1E05A0730F4A8E0BA2EE22CAFE00A
:10056000AA2E1DC0403DA2E05A0730F4A4E0BA2EE6
:10057000E22CAEE1AA2E13C0403AA5E05A0730F4AF
:10058000A2E0BA2EE22CACE3AA2E09C04839A8E0BA
:100590005A0728F4A1E0BA2EE22CA8E7AA2EC42E0E
:1005A000A0918A00CA1AD52EA0918B00DA0ADD200C
:1005B0002AF4AFEFC094D094CA1ADA0A20928C00C1
:1005C000CA14DE0418F4A1E0A0938C0040938A00C2
:1005D00050938B0040918800509189004093860091
:1005E00050938700A09164004A1BA09165005A0BAC
:1005F00094FD7CC093FD7AC092FD76C056954795D8
:1006000091FD72C05695479590FD6EC0D52EC42EB3
:10061000D694C79461FD0CC0AC2DAC51AD2DA24059
:1006200008F07BC0DD2021F4AC2DA85C08F475C077
:10063000A0E0EA2E97FD08C0E090C200A091B400AF
:10064000A33011F4E090CA00AAEFEA0EF22CF21CDB
:10065000CE18DF084FB74170A091B400A330A9F4C1
:10066000442329F095FD11C0F894906204C095FFD1
:100670000CC0F8949F7D9598AC98C098AB98AD98B5
:10068000949871FD01C060687894442369F0A0914A
:10069000B400A33031F4AFEFC094D094CA1ADA0A90
:1006A00003C040E050E022C0A091B400A33049F460
:1006B000CC0CDD1CA5E0CA1AD20818F4A0E0CA2EA2
:1006C000D22CAFEFCA16D20418F04FEF50E00EC094
:1006D000F090A700CF9C412D000C441F50E008F083
:1006E00012C04FEF50E00FC05695479594FF07C0DA
:1006F000552309F04FEFA42FA6954A0F521D4F3FE7
:10070000520508F04FEF40938D00816061FF05C0F6
:10071000AFE1A095A923AB299A2FA8E1A093660089
:10072000A92FAF7119F4AAE0A093660061FD04C07F
:10073000A92FAF7109F08F7EA6E0A0936700A92FC3
:10074000AF7119F4AAE0A0936700F894A9B7A1606B
:10075000A9BF84FF02C0A0E4ABBF3FBE189511E063
:100760000AC013E008C01AE006C01EE104C014E687
:1007700002C018EC00C005E1BB27BA95F1F70A9555
:10078000D9F71A95C1F708952AE338E709C020E39D
:100790003CE806C02AE234EB03C025E238EC00C096
:1007A000652CB1E05B2E12E095FD9F7D95FF906278
:1007B000BB27AD98BA95F1F7552009F0AC9ABA95D8
:1007C000F1F7AC98BA95F1F7AD9ABA95F1F75520D3
:1007D00021F095FF959A95FDC09AB091A800BA9521
:1007E000F1F795FF959895FDC098B7E8BA95F1F7A0
:1007F0001A95D1F6022FB22FBA95F1F70A95D9F7CB
:100800003A9571F6AD98562C0895221B39E0001FD9
:100810003A9509F40895221F211B18F4210F88949A
:10082000F6CF0894F4CF622C722CB0E08894B39584
:10083000221F331FE0F7379527958894912E802E3D
:10084000020B130B10F4192D082D10F4889401C01D
:100850000894661C771CBA9571F7172D062D08951C
:10086000322D11232AF43A9500951095031B130B92
:10087000F894029F712C002D129F912C802C78945B
:10088000780C172D921C292DB4E06B2E2695179508
:1008900007956A94D9F7332321F000951095031B2F
:1008A000130B08950091AE000430A1F1B0918D00BA
:1008B000B15008F010C0B0916100B0936300209275
:1008C0007700209278002092790020927A0020927E
:1008D0007B006F7B1FC06090AE006064B0916100D0
:1008E000B093620008E317EC20917300309174001C
:1008F00036952795B62DBA9541F036952795B62DA4
:10090000BA95BA9511F0369527958DDF009377004B
:1009100010937800089566FF1BC000917700B09196
:1009200062000B1B10917800120928F40038BFEF09
:100930001B0740F009C00F37120508F405C00FE788
:1009400010E002C000E81FEF00937C0010937D00D0
:10095000089566FF39C000917C00B09179000B0FBB
:1009600010917D00B0917A001B1F20E030917D0036
:1009700033230AF42A95B0917B002B1F1AF4203FF1
:1009800040F00AC02F3008F407C00FEF1FEF2FE030
:1009900003C000E010E020EF30916300B0919200BE
:1009A0003B1718F4332331F009C0B0917D00BB230D
:1009B0005AF004C0B0917D00BB2332F4009379005B
:1009C00010937A0020937B00089566FF2FC020913A
:1009D000CD0000917C00000F10917D00111F40DFC1
:1009E00011232AF40038BFEF1B0740F009C00F376E
:1009F000120508F405C00FE710E002C000E81FEF81
:100A0000002352F0B0916200B01B0B2F18F00130A0
:100A100008F00AC001E008C000950F5FB0916200C5
:100A20000B0F08F001C00FEF00937E00089566FFE2
:100A30002DC02091CE0000917A0010917B0010DF34
:100A400011232AF40130BFEF1B0740F009C00F3F0C
:100A5000120508F405C00FEF10E002C001E01FEF1F
:100A6000112352F0B0917E00B01B0B2F18F0013013
:100A700008F00AC000E008C000950F5FB0917E004A
:100A80000B0F08F001C00FEF0093630008950FEF04
:100A9000677FB72FB670E9F46860B0917400B83022
:100AA00008F0677FB0917400A1F00FEF109174000F
:100AB000ACDEF894B09170000B9F112D002D78944E
:100AC000112309F00FEFB09195000B1710F400916E
:100AD00095000093940008951AD374FFB2E074FD5A
:100AE000B1E0B7B9B6B1B068B064B6B938DE74FF7A
:100AF000B2E074FDB1E0B7B9B6B1B068B064B6B9F0
:100B0000B6B1B6FDFDCF04B115B1B6B1BF77B6B978
:100B100043D324E72093A30030E03093A400732E46
:100B20007694622E6694620E731E262D372D021760
:100B3000130778F08090A300B4E7B80DB093A3003A
:100B40008090A400B0E0B81DB093A400260D371D1E
:100B5000EECF8090A3009090A4001091A400169571
:100B60000091A300079516950795B091A300B00FCB
:100B7000B093A100B091A400B11FB093A20023E0F4
:100B8000169507952A95E1F72091AF002A9529F44B
:100B90002092A3002092A4000AC02A9521F0800E82
:100BA000911E2A95E1F78092A3009092A4000895E7
:100BB0002091AF00B6B1B6FDFBCF04B115B1B6B10F
:100BC000BF77B6B9B091A500B395B093A500B83082
:100BD00060F12092A500B091CC00BB2321F111233C
:100BE00029F0B091A600BF3F61F009C0B091A60006
:100BF0000B1739F020F4BB2321F0BA9502C0B3954E
:100C0000E1F300919200B093A600B13A50F400ECE9
:100C1000B43938F400E8B73820F400E4BA3708F4FF
:100C200000E0009392007F7E0895213099F00F3FFD
:100C3000B3E01B0778F4B091A3000B17B091A400A8
:100C40001B0740F4B0919200BB23A9F0BA95B09372
:100C5000920011C0B0919200BF3F69F0B395B0937C
:100C60009200B091B400B33031F4B0919200BC5F07
:100C700010F4B093920000919200B0916300B01B09
:100C800010F400916300B09193000B1750F00091A5
:100C90009300B0919300BF3F21F0B0919300B093C7
:100CA0009200B091AE00B43009F406C0B091940047
:100CB0000B1708F00B2F502EB091A500B73009F498
:100CC0007061089502E3F894B091D0000B9F012D5C
:100CD000000C001F7894B09192000B1710F0009157
:100CE00092000093610000936300502E00939500E2
:100CF000089520927300B8E0B09374000895209195
:100D0000800030918100F8940CB51DB5200F311F83
:100D10003BBD2ABD6160B0E1B8BF789420917100FD
:100D2000309172000093710010937200021B130B3C
:100D30002091730030917400622E732EB4E08B2EDC
:100D4000B2E09B2EB0917400B43010F08A949A9463
:100D5000B83010F08A949A94769467948A94E1F764
:100D600026193709992021F0169507959A94E1F7ED
:100D7000200F311F209373003093740008F0089502
:100D8000BFEFB0937300B093740008952091820078
:100D900030918300F8940CB51DB5020F131F1BBDD5
:100DA0000ABD6160B0E1B8BF7894089560FDFECFE0
:100DB000EDDF0895B091BE0000916E00023808F09A
:100DC000B395003A08F0B395B63008F0B5E09B2E25
:100DD000BCE08B2EB0917400B33030F483948394D4
:100DE00082FF02C083948394B23030F4839483945E
:100DF00082FF02C08394839471FF03C0B3E09B2EF3
:100E0000822C109174000091730024E016950795D0
:100E10002A95E1F70819120928F0B02FB250B12F26
:100E2000B20910F402E010E0312F202F712E602E55
:100E300076946794B92DB330E9F0B0FD05C0060D86
:100E4000171D262D372D06C0000F111F0250120945
:100E500022E030E0B92DB33068F020938400309365
:100E60008500009380001093810060928200709250
:100E700083000895009384001093850020938000E0
:100E8000309381006092820070928300089560FD2B
:100E9000FECF20918200220F30918300331FB72FA5
:100EA000B67021F02091730030917400F8940CB565
:100EB0001DB5020F131F1BBD0ABD6160B0E1B8BFB5
:100EC0007894089560612092760020E004C060610B
:100ED0002092760020E2B72FB67009F06F7E7894EA
:100EE00060FD05C0B0917600BB2309F0089501E0D4
:100EF00063FF0AC0B0917400B33008F002E0B09113
:100F00007400B63008F003E071FF01C006E060FD38
:100F100006C0B0917600BB2311F0789408951AE0D2
:100F200083FF1AE0789400000000F89462FD03C08B
:100F300014E183FF14E171FF01C018E7B4B53091EB
:100F40009900B31BB10B18F3B0917600B395B09331
:100F50007600B5E03B2F6B2E722CB8B1B072B21791
:100F600009F073943A95C9F77394761488F464FF82
:100F7000B2CF6F7E3CB56DB47090730080907400FA
:100F8000370D681C6BBC3ABD6160B0E1B8BFA3CF40
:100F900064FDA1CF0A9509F0BACF7894089571FF46
:100FA0000AC0B0916D00B395B0936D0060FD0CC0A8
:100FB00020926D0009C060FD07C064FD05C067FD9B
:100FC00003C0BF91BF9159C408952091840030910E
:100FD0008500F8940CB51DB5020F131F1BBD0ABD8B
:100FE0006160B0E1B8BF78940895EFDF00E063FF7F
:100FF00003C064FF01C001E0F89410916E00B7E0F7
:101000001B9F212D102D7894200F2695179526953E
:1010100017952695179510936E00183718F4B8E7B2
:10102000B0936E0000916E00B0916F000B1720F02E
:1010300060629598AC98C09860FDFECF0895F894D2
:10104000AB98AD98949882FF07C0E0E0F1E073FFA1
:1010500003C0B5E0BA95F1F795FFAB9A95FD949A68
:10106000B2E0B093750089C0F89495FFC09895FDE3
:10107000959882FF0DC0E0EFF0E073FF0BC0AD98D4
:1010800095FF949895FDAB98B5E0BA95F1F702C03D
:10109000EAEAF0E062FF03C0552009F0AC9AB3E041
:1010A000B09375006AC0F894AB98AD98949882FF9D
:1010B00007C0E0EEF0E073FF03C0B5E0BA95F1F7CA
:1010C00095FF949A95FDAB9AB4E0B093750055C026
:1010D000F894AC9882FF0DC0E0EDF0E073FF0BC018
:1010E00095FFAB9895FD9498AD98B5E0BA95F1F75A
:1010F00002C0E2EAF0E062FF06C0552021F095FF51
:10110000959A95FDC09AB5E0B093750036C0F894F5
:10111000AB98AD98949882FF07C0EDEBF0E073FFB9
:1011200003C0B5E0BA95F1F7AD9AB6E0B09375009B
:1011300024C0F89495FF959895FDC09882FF10C043
:10114000E3E1F1E073FF0EC095FFAB9895FD949835
:1011500095FF949895FDAB98B5E0BA95F1F702C06C
:10116000E2EBF0E062FF06C0552021F095FFC09A47
:1011700095FD959AB1E0B093750067FF0AC00CD059
:10118000B5E0BA95F1F7B5E0BA95F1F7AB9AAD9A3B
:10119000949A6F7D7894089521EA30E0F90195984A
:1011A000AC98C098AB98AD9894986B7F0895ACEAD2
:1011B000B0E009E00D9309E00D9304E00D9301E028
:1011C0000D9303E00D930FEF0D9309E00D9301E0F4
:1011D0000D9301E00D9301E00D93A8EBB0E001E069
:1011E0000D930FEF0D930D930FEF0D930D930D9343
:1011F00003E00D9306E00D930FEF0D930D9305E2C1
:101200000D9300ED0D9308E20D9300E50D9304E0BE
:101210000D930DE00D9302E00D9300E00D930AE7AE
:101220000D930FEF0D9301E00D9308952091BF00F2
:1012300009E011E0223011F405E011E0233011F44F
:1012400005E012E0243011F405E013E0253011F43C
:1012500009E017E0263011F400E010E000939F0051
:101260001093A0002091B3008B7F777FB091B400E2
:10127000B33019F09F7DB1FD90629F7BB091B500B6
:10128000B1FD9064B22FB23011F0886001C0877F49
:101290000895ECE1F0E00091AC000A95E00FF21D3A
:1012A000B491B093CD000091AD000A95E00FF21D0E
:1012B000B491B093CE0070DF0895EAE2F0E00091BF
:1012C000C7000A95E00FF21DB491B093CF0064DF20
:1012D0000895E8E3F0E00091B2000A95E00FF21DF6
:1012E000B491B093D00058DF08950895B091C8002C
:1012F0000FEF1CE0B23011F400EA1AE0B33011F441
:1013000002E815E000936F001093700008950895AF
:101310002091C2003091C30097FF02C020E03FEF50
:10132000B32FB21B6B2EB25810F4B2E86B2E00E054
:101330000395609EB12DB058D8F30093A70008958F
:10134000F894E3E0F0E0B9E0B7BFB491B078C1F34E
:10135000F894A895B1B5B861B1BDB0E0B1BDB4E045
:10136000BEBFBFE5BDBF18DFB0E0B8BBB1E1B7BBE2
:10137000B0E0B5BBB8E3B4BBB0E0B2BBB0E3B1BB67
:101380002224A0E0B0E02D92AA31E9F7A0E6B0E077
:101390000FEF2D920A95E9F70ADF8FD247DF79DF49
:1013A0008CDF97DFA2DFA2DFB2DFB2DF0091C400E3
:1013B0000093A800F1DEB2E0B3BFB2E0BEBDB2E080
:1013C000B5BDF894D6D9E0D9D0D9E1D9CED9E2D9F2
:1013D000CCD9CFD9CED9CBD9B1E5B8BFB9BFB0B789
:1013E000B860B0BFB6B1B460B6B9B9D9789474DB9F
:1013F000B0E4BBBFBB27B064BABF8D7FBAD9B1E040
:10140000B0936900626025E0B0918C00BB2309F4C1
:1014100025E0A7D9B0918D00B230A8F3B92FBF71E4
:1014200000918F0000938E00B0938F00B01759F792
:101430002A9551F76D7F96FFB3E096FDB2E0B5BFF8
:10144000BB27B064BABF8D7F92D98BD902E0B92F88
:10145000BF7109F400E0B0918D00B017B0F3F894BB
:1014600093D992D991D9789484D920927F00B09160
:10147000B400B33009F472C074D9B091B800B1307F
:1014800008F46CC0B0916900B13008F467C0B92F9E
:10149000BF71C1F0B0918D00BF3F08F45FC0F894F8
:1014A0007CD9789464D9B0918D00B130C0F7F894AC
:1014B0006BD959D969D978945AD9B0918D00BF3F69
:1014C000B0F3C4C2B3E09B2E9068F89421DF789407
:1014D0004ED9F8949F771CDF80908D00B0918D00DD
:1014E000BF37789408F442C03AD9F89456D9789422
:1014F0009A9451F7B82DB550B093C3003AD9F894E7
:1015000009D277D27894BAE09B2E9068F89400DFE5
:1015100078942DD9F8949F77FBDE80908D00B09160
:101520008D00BF37789478F71AD9F8942DD91BD944
:101530002BD978949A9449F7B82DBB5FB093C20029
:1015400018D9F894E7D164D2789411D9F894E0DEF0
:101550007894B0918D00BF3FC0F378C200918D00A8
:10156000B0917F000B1710F000937F0000D901E0CD
:10157000B091B400B35009F405E0B0918D00B017FC
:1015800008F075CFF89409D908D907D97894F1D81B
:101590002092690020926A0020926B00B0916A004C
:1015A000B395B0936A00BF3F69F5B0916B00B395F6
:1015B000B0936B00B091C60009E1BA9559F002E30F
:1015C000BA9541F00DE7BA9529F00AEFBA9511F0F6
:1015D00020926B00B0916B00B017A0F0B0916B003F
:1015E000BA95B0936B00B4EBB0936A00B091C500AC
:1015F000B093A800F894D1D87894B091C400B09377
:10160000A800B5D8B0D8B0916600BB2321F4B92F9B
:10161000BF7109F4F7CEB0918D00B63008F4BECF9B
:10162000B091B400B35009F0A2D8B0916600BB23CA
:1016300009F4E8CEF894B0DD2092610020926200B7
:1016400020926300522C7894B091B100B093960030
:1016500020927700209278002092790020927A00E0
:1016600020927B002092A50060E070E020926E0046
:1016700040DBB8E0B093A500706171D874FFB2E0B0
:1016800074FDB1E0B7B9B6B1B068B064B6B9B6B17F
:10169000B6FDFDCF04B115B1B6B1BF77B6B9112310
:1016A00009F00FEF0093A60083DAB8E0B093A5002D
:1016B00070618090B300B2E0B093B300B7DD809268
:1016C000B300F894BFEFB0939200FCDAB0916100E0
:1016D000B0939200B0939300B09394007894B1E0EB
:1016E000B0936100B09363005B2EB0939B00B09108
:1016F0009100B0939A007160726020926D0007DDD6
:1017000018DDFDDAF6DA56DB04C090DD2092A50084
:101710007F7E95FFB0E095FDB6E0B7B9D8DB3FDC42
:1017200054DCC0D862DC8BDCEADA40DB43DBAFDBC5
:10173000B7E0B7B9C7DB33DC48DCEDD8A8D955DC56
:1017400093DCDDDA33DB36DBA2DB95FFB6E095FD1B
:10175000B0E0B7B9BCDB23DC38DCFBD846DCA3DC6B
:10176000CEDA24DB27DB93DB95FFB0E095FDB6E016
:10177000B7B9A8DB14DC29DC28D937DCA9DCBFDA4F
:1017800015DB18DB84DBB7E0B7B9A1DB08DC1DDCB7
:101790004ED92BDCBCDCB3DA09DB0CDB78DB95FF44
:1017A000B6E095FDB0E0B7B98DDB74FFB2E074FD33
:1017B000B1E0B7B9B6B1B068B064B6B9F0DB05DC7A
:1017C00014DCB7DC9CDAF2DAF5DAF2D960DB71FF0F
:1017D0002EC067FD2CC0B0919500B0939200B093DD
:1017E0009300B0919100B0939A00B1E0B0939B0048
:1017F00014E624E1B0916D00B11798F07D7F74601C
:1018000020936C00B091B400B33051F4B0919500C6
:10181000B0939200BFEFB0939300B0E2B093940006
:1018200006C0B0918D00B13008F073CF26C072FFB2
:1018300010C067FD0EC0B0916C00BA9511F47B7FAB
:1018400064CFB0936C00B0918D00B13008F061CFDF
:1018500014C0B0919000BA3F80F4B92FBF7121F449
:10186000B0916600BB2349F0B091740000EF67FFB0
:1018700001C000E6B01708F44CCFF8948DDC8090DE
:10188000B300B2E0B093B300D1DC8092B3002092F9
:1018900061002092620020926300522C20929600F8
:1018A0007E7F78945CD778DCB92FBF7129F4B09132
:1018B0006600BB2309F4A6CD6DCEEDE0F0E023D0A9
:1018C000053509F01BC0EEE0F0E01DD00A3A09F042
:1018D00015C03AE0ACEAB0E0E3E0F0E014D00D93DC
:1018E00031963A95D9F735E1A8EBB0E0EFE0F0E0BA
:1018F0000AD00D9331963A95D9F702C058DC0AD038
:10190000E4E2F0E00895E199FECFEEBBFFBBE09A80
:101910000DB308951ED03AE0ACEAB0E0E3E0F0E0A9
:101920000D910FD031963A95D9F735E1A8EBB0E09B
:10193000EFE0F0E00D9105D031963A95D9F712D04D
:101940000895E199FECF0DBBEEBBFFBBE29AE19A91
:101950000895EDE0F0E00FEFF4DFEEE0F0E00FEFE0
:10196000F0DF0895EDE0F0E005E5EBDFEEE0F0E01C
:101970000AEAE7DF08953091A9000091AA0031300A
:1019800011F40093AC00323011F40093AD00333009
:1019900011F40093AE00343011F40093B0003530F0
:1019A00011F40093AF00363011F40093B2003730D9
:1019B00011F40093BE00383011F40093C7003930A1
:1019C00011F40093BF003A3011F40093B3003B30A0
:1019D00011F40093C8003C3011F40093B4003D3082
:1019E00011F40093B500089525E0C3D62A95E9F7D0
:1019F0000895CAD6CCD6CED6D0D6B5D6C5D6C7D6FB
:101A0000C9D6CBD6B0D6C0D6C2D6C4D6C6D608950F
:101A1000C4D6C0D6BCD6B8D6A6D6BFD6BBD6B7D647
:101A2000B3D6A1D6BAD6B6D6B2D6AED608958090E1
:101A3000A9009090AA00A8D6A7D6A6D694D68A9434
:101A4000D1F7ABD690D69A94E1F70895F894D1DF08
:101A50007894CADFC9DFB1E0B093A900B1E0B093D8
:101A6000AA002092AB00F894E2DF7894B5E06B2EE8
:101A700070908D007ED6B0918D007B16C9F7B13085
:101A800018F0BF3F40F107C076DFF89443DFB1DFC5
:101A9000B8E0B1BDA9DF6A9459F7B091AB00B39536
:101AA000B093AB00B33008F4DECF9EDFB091AA0054
:101AB000B395B093AA00F894B091A900BA95E6E462
:101AC000F0E0EB0FF21D049178940395B091AA0019
:101AD000B01708F4C6CF88DF87DFB091A900B395AF
:101AE000B093A900B091A900BE3008F4B7CF5FDB76
:0A1AF000F89410DFB8E0B1BD77DF15
:00000001FF
